:100000006BC0D5C184C083C082C081C080C07FC0A6
:100010007EC07DC07CC07BC07AC079C078C077C00C
:1000200076C075C074C062C45EC456C451C457C49F
:1000300058C46EC46BC44EC44DC46CC46DC44AC4B1
:1000400049C45DC459C454C455C444C443C442C41F
:1000500041C457C459C40403090418037200610061
:10006000700068006E00650074002E006E00650070
:1000700074001E03320061007800650073003100D7
:10008000360062007500740074006F006E0073002B
:100090000A03310030003000300005010905A101DC
:1000A0000901A10009300931150026FF00750895E6
:1000B000028102C0050919012910150025017501E9
:1000C00095108102C0120101010000000881179CF7
:1000D0000A0001010203010011241FBECFE5D4E094
:1000E000DEBFCDBF10E0A0E6B0E0E6E1FCE002C07C
:1000F00005900D92AA39B107D9F710E0AAE9B0E04E
:1001000001C01D92AA3EB107E1F719D383C578CF8C
:1001100085B7836085BF8BB780648BBF83EC80938A
:10012000C00008950F931F93CF93DF939091D00059
:1001300019160CF0A5C02091CD008091CC008D3215
:1001400009F096C08AE5809361009B3009F090C069
:10015000C0EED0E0C21BD1098881807609F079C059
:100160002EEB30E01092BE008981882341F410927A
:10017000BF003093CF002093CE0092E06DC0853059
:1001800021F48A818093D10062C0863009F043C097
:100190008B818130E1F1823019F4CE016BD25BC0EA
:1001A000833049F58A81882341F486E590E0909375
:1001B000CF008093CE0094E052C0813041F48AE5B4
:1001C00090E09093CF008093CE0098E148C08230B9
:1001D00041F482E790E09093CF008093CE009EE1BF
:1001E0003EC08330D9F580E990E09093CF008093B2
:1001F000CE009CE034C0813241F48DEA90E09093CF
:10020000CF008093CE0099E02AC0823239F5CE012A
:1002100031D2982F24C0883039F483ED90E0909348
:10022000CF008093CE000CC0893021F48A81809366
:10023000D3000DC08A3031F43093CF002093CE002C
:1002400091E00AC08B3019F483EC8093C00090E0F9
:1002500003C0CE0140D2982F20E802C090E020ECED
:100260008F81882339F48E81891720F4982F02C05A
:1002700090E020E820939A00909360001092D000C4
:100280008091610084FF45C0809160008F3F09F438
:1002900040C0182F893008F018E0811B809360005F
:1002A00080919A0080FF02C003EC01C00BE48F5FD5
:1002B00080939A002091CE003091CF0086FD05C03A
:1002C000912FF901A6EBB0E00DC0912FF901A6EB3B
:1002D000B0E003C084918D9331969150D8F704C05B
:1002E00081918D939150E0F7C901810F911D9093F9
:1002F000CF008093CE00612F86EB90E054D0183071
:1003000019F08FEF809360000093B5001C5F10938D
:1003100061009AE080B3857031F49150D9F7109262
:10032000D1001092CB00DF91CF911F910F910895D2
:100330001F93DC01162F8091620084FF07C080911B
:10034000C00098E889278093C00003C08AE58093A5
:100350006200912FE1ECF0E002C08D918193915009
:10036000E0F7612F81EC90E01ED01C5F10936200DB
:100370001F910895A82FB92F8FEF9FEF41E050EA0A
:10038000615070F02D9138E0722F782796958795FF
:10039000269570FF02C0842795273A95A9F7F0CFDC
:1003A000809590950895E6DF8D939D930895CF9362
:1003B000CFB7CF93809BFECF809B09C0809B07C0A7
:1003C000809B05C0809B03C0809B01C09EC0DF93C3
:1003D000C091CD00DD27CC52DF4F809B02C0DF9162
:1003E000EBCF2F930F931F9300B32FEF00FB20F958
:1003F0004F933F9310B34FEF012700FB21F93BE0F0
:1004000031C04E7F012F10B3216028C0102F4D7FC7
:100410002260000000B329C04B7F2460012F000040
:1004200010B32BC010B3477F28602AC04F7E00B3A3
:1004300020612CC04F7D10B320622FC04F7B00B3D2
:10044000206432C0422700B349934FEF00001027C9
:1004500010FB20F910B31570A9F1297F91F2012743
:1004600000FB21F900B3237F89F23150F0F110270E
:1004700010FB22F910B3277E79F2012700FB23F944
:100480002F7C81F200B3102710FB24F92F7971F231
:1004900000C010B3012700FB25F92F7359F200C0EB
:1004A00000B3102710FB26F9223040F200C010B331
:1004B000012700FB27F9243028F64F77206810B376
:1004C0000000F9CF3B503195333010E41ABFB8F03B
:1004D000C31BD0400881033C41F10B3431F1198139
:1004E000412F1F772091CB00121731F4093691F17B
:1004F0000D3279F0013E69F022272093D2003F911E
:100500004F911F910F912F91DF91CF91CFBFCF913D
:1005100018950093D2003F914F911F910F912F9109
:10052000DF91CAB7C6FD46CFF0CF0091D2000023BD
:1005300031F31091D0001123A1F53430A2F13093A2
:10054000D0000093CC001091CD003BE0311B3093E4
:10055000CD0029C00091D00001301CF50AE547FD0F
:1005600009C03091610034FD20C000936100C5EBEB
:10057000D0E01FC03091620034FD17C000936200CC
:10058000C0ECD0E016C0052710E002BB1FC0052755
:1005900022C0052727C005272CC0052710E002BB75
:1005A00033C04AE503C042ED01C0432FC4E1D0E0AF
:1005B00032E011B31560909A02B311BB5F9355E01E
:1005C00020E820FF052702BB279517951C3FD8F68A
:1005D00020FF0527279502BB17951C3FC0F620FF7B
:1005E00005272795179502BB1C3F98F620FF052786
:1005F000279517951C3F02BB70F600C0499120FF5C
:10060000052702BB279517951C3F38F620FF0527C5
:10061000279502BB17951C3F38F520FF0527279526
:10062000179502BB1C3F10F520FF0527279517954E
:100630001C3F02BBE8F4242F3A9519F60A7F5F911C
:1006400002BB00C01091D100C651D04011F01093F0
:10065000CB0010E41ABF016011B31A7F402F4A7F0C
:1006600002BB11BB42BB4BCF0527D3CF0527D8CF49
:100670000527DDCFFC018081807651F581818630B0
:1006800039F583818230D9F0823269F0813001F509
:1006900080919F009091A0009093CF008093CE0016
:1006A0008091A1000AC080919C0090919D00909340
:1006B000CF008093CE0080919E009927089583E615
:1006C00090E09093CF008093CE0082E290E0089576
:1006D00080E090E00895FC0124EA30E03093CF0000
:1006E0002093CE0080818076803231F58181813007
:1006F00081F4E091A200F091A3000088F189E02D3F
:10070000C9010995E091A200F091A3008081992789
:100710000895823049F48AEA90E09093CF00809364
:10072000CE0081E090E008958A3031F48381809397
:10073000AA0080E090E0089580E090E00895CFE581
:10074000D4E0DEBFCDBFB89A87B3897F87BB88B3BB
:10075000866088BBC09880E395E70197F1F786B380
:1007600006D2FC019093A3008093A200848195811E
:1007700090939D0080939C00828180939E00808551
:100780009185009731F09093A00080939F0086811F
:1007900007C085EC90E09093A00080939F002AD240
:1007A0008093A10080919E0080937C0014BA8FEF0B
:1007B00085BB88EF82BB85E081BB11BA83BF8FE028
:1007C00085BD84EC83BDE091A200F091A30002847A
:1007D000F385E02D09959CDC789400E011E0FF247E
:1007E000C4EAD0E001C010E0A8959CDC112341F0E0
:1007F000E091A200F091A3000484F585E02D099515
:1008000008B600FE0EC081E088BF8091AA00882350
:1008100041F094E09F1518F0F82E01E002C08BEF34
:10082000F80E08B607FE18C080E888BF0023B1F4B0
:10083000E091A200F091A3000484F585E02D0995D4
:10084000E091A200F091A3000684F785E02D0995C0
:10085000882349F201E002C0002329F2809162005E
:1008600084FFC1CFE091A200F091A3000088F1893C
:10087000E02DCE010995E091A200F091A3006081E6
:10088000CE0156DD00E0AFCFCF93DF93EC019B01AB
:1008900087B3817C87BB88B38E6388BB15BA80E23F
:1008A00084BB8FE185BB88EB9BE00197F1F783B3B5
:1008B00080959927AA27BB278F719070A070B07080
:1008C000FC013297E831F10528F4ED5EFF4F099401
:1008D0009EEF18C090E001C09EEF80E01FC09EEF29
:1008E0000CC09EEF01C09FEF8EEF18C090E0FCCFD0
:1008F00091E0FACF92E0F8CF92E08FEF0FC092E054
:10090000ECCF92E081E00AC092E007C091E005C020
:1009100090E003C09FEF01C09EEF82E08883F90161
:100920009083DF91CF9108958F3F99F08F3F09F029
:100930001CF48E3F41F40AC0813071F0823019F40A
:100940008FEF90E0089580E890E0089580E090E0D7
:10095000089580E490E0089580EC90E008950F936E
:100960001F93CF93DF93CDB7DEB724970FB6F894DC
:10097000DEBF0FBECDBFBE016C5F7F4FCE010396C1
:1009800083DF84B3817E84BB85B38E6185BB88B3EE
:10099000877C88BB87B3886387BBE8EBFBE0CF012C
:1009A0000197F1F723B3269585B3817E85BB84B388
:1009B0008E6184BB88B3877C88BB87B3877C87BB09
:1009C00088B3886388BB3197F1F786B3869586959F
:1009D0008695809520958770992734E0880F991F18
:1009E0003A95E1F72F703327822B932B82329105B2
:1009F00009F440C08332910594F48431910589F162
:100A00008531910534F48131910529F1429701F541
:100A100025C08831910541F18197D1F428C08134F6
:100A2000910589F18234910534F48432910529F1DC
:100A3000889771F425C08434910559F18834910563
:100A400021F08234910521F421C000E210E023C09E
:100A500000E010E020C000E010E11DC000E012E066
:100A60001AC000E410E017C008E010E014C000E075
:100A700010E211C000E014E00EC000E810E00BC06E
:100A800000E110E008C000E010E405C000E018E05C
:100A900002C000E011E015BA14BA8FEF85BB18BA96
:100AA00088E087BB88B3806388BBE8EBFBE0CF01BD
:100AB0000197F1F786B38073992784FF046085FF5F
:100AC000016018BA80E187BBC59A3197F1F7B59BF1
:100AD0000260C801887F892B21F08091AC00898356
:100AE00014C0BE016E5F7F4FCE010196CDDE9981AD
:100AF0008B81981721F08091AC00898302C090937C
:100B0000AC009A818C81981721F08091AB008A8388
:100B100002C09093AB0089812FE38202C0011124AF
:100B200080588093AD008A818202C00111248058D0
:100B30008093AE000093AF00812F99278093B0007F
:100B400024960FB6F894DEBF0FBECDBFDF91CF91D4
:100B50001F910F9108951F931FB7F89414BA17BAF5
:100B60008FEF85BB88BBFBDE1FBF1F9108958AE90D
:100B700090E090938A008093890085E890E0089542
:100B8000FC01892B61F08091AD009091AE00A091A5
:100B9000AF00B091B00080839183A283B383809132
:100BA000AD009091AE00A091AF00B091B0008093E5
:100BB000B1009093B200A093B300B093B400089535
:100BC0008091970090919800892B39F010929800AD
:100BD0001092970021E030E00BC044E050E061EB60
:100BE00070E08DEA90E009D0282F332727FD30955B
:100BF000C901089582E190E00895FB01DC0104C081
:100C00008D910190801921F441505040C8F7881B04
:060C1000990B0895FFCFCF
:100C1600FF5A5A090222000101008032090400002D
:100C2600010300000009210101000122000007055F
:100C3600810308000A04002B00000000000000AB3E
:0A0C460005AF04E005C00501000041
:00000001FF
